:03F0000002F00813
:03F0610002F003B7
:05F0030012F10F80FE78
:0DF0640090DF10E090FDF0F090DF0FE090E5
:0EF07100FDF1F090DF0EE090FDF2F090DF0D6B
:0EF07F00E090FDF3F090DF0CE090FDF4F02245
:0DF08D0090FDF0E090DF10F090FDF1E090BC
:0EF09A00DF0FF090FDF2E090DF0EF090FDF33E
:0EF0A800E090DF0DF090FDF4E090DF0CF02220
:03F0B60053BEFB4B
:08F0B900E5BE30E6FB53C6B8CA
:0EF0C100E5C620E6FB43BE0490DF0C7486F02B
:0DF0CF0090DF0D7483F090DF0E7430F09030
:0CF0DC00DF0F7422F090DF1074F8F022B7
:04F0E800AA82AB83CA
:05F0EC001ABAFF011B30
:0EF0F100C3E49A74808BF063F08095F0500FAA
:04F0FF007CB07D0460
:05F103001CBCFF011D12
:06F10800EC4D70F780DE03
:01F10E0022DE
:09F10F0090FE00E0C2A812F064B9
:03F1180075E1049A
:0EF11B0090DF3BE0FABA01F812F08D12F145D8
:09F1290012F0B675E10475E10372
:0EF1320090DF3BE0FA53021FBA13F590000A7B
:05F1400012F0E880D38D
:02F145007A004E
:03F14700BA4000CB
:0DF14A00500B8A827583FE74FFF00A80F07E
:05F15700C2A875E104EF
:0BF15C0090DF3BE0FABA01F875E10219
:0DF1670090DF3BE0FABA0DF890DF02E09077
:05F17400FE00F07A012D
:03F17900BA0300D6
:02F17C0050132E
:05F17E0010890280FB76
:0EF183008A030A8B827583FEE5D9FBF080E8D3
:04F1910075E10422FE
:06F03700E478FFF6D8FDAD
:08F015007900E94400601B7A58
:05F01D000090F199785C
:03F02200007593E3
:0AF0250000E493F2A308B80002050E
:08F02F0093D9F4DAF27593FFA6
:08F03D007800E84400600A7944
:03F04500007593C0
:06F0480000E4F309D8FC0E
:08F04E007800E84400600C7931
:0BF0560000900000E4F0A3D8FCD9FA01
:03F0080075810708
:0AF00B0012F195E582600302F003A4
:04F19500758200225D
:00000001FF
